:104E3A0000000501013C0200000400FA0301FA0522
:104E4A0000020A0A5A0B000F0C00FA0D00030E00AA
:104E5A00030F0132100096120132130AFA140102EA
:104E6A0015010217010A18010A1905321A010A1B4B
:104E7A00010A1C053223011E2400642A00FA2B00B1
:104E8A00FA2C50782D003C2E00462F001E3000646C
:104E9A003250783300003432FA350164360164370F
:104EAA000050380A643C00643E003C3F000140FF69
:104EBA00FF411450420A5A430AC844053245007851
:104ECA004600FA47013A4802024C00FA4EFFFF50E8
:104EDA000505510596521432530B28540A96560169
:104EEA0001570546580001590A465A32FA5B010A27
:104EFA005C14325E000A5F00FE61FFFF64031C66F9
:104F0A0000016701036A0A3C6B00006C3296780163
:104F1A0032790132FAFAFA0065006F0079008300EB
:104F2A008D009700A100AC00B600C000CA00D400F2
:104F3A00DE00E800F2005B0063006A0072007A009B
:104F4A008200890091009900A100A800B000B80071
:104F5A00BF00C700CF00D600DF00E600EE00F60073
:104F6A00400046004C00520059005F0065006B008B
:104F7A00710077007D00830089008F0095009C00F6
:104F8A00A200A800AE00B400BA00C000C600CC005F
:0B4F9A00D200D900DF00E500EB00F1C1
:10009E00AE33AF3474068E048F05FF1200858C3597
:1000AE008D36AE33AF3474068E048F05FF12522890
:1000BE008C338D34E534453360137406C39534FFA9
:1000CE00E49533FE8E338F347835125274E550A892
:1000DE0035B80015D395364010E550C39536FFE47C
:1000EE009535FE8E358F368010E550243CC39536FF
:1000FE00FFE49535FE8E358F36AE35AF36743B6FD9
:10010E004E6006743C6F4E701AAE35AF36743B6F50
:10011E004E7005755001800375500275363A75356F
:10012E000080037550002290009AE0B40104C20BC7
:10013E008002D20B90009BE0B40104C20C8002D26C
:10014E000C9000D8E075F0DCA4FFAEF0740A8E04BB
:10015E008F05FF1200859007C0ECF0A3EDF0A2080A
:10016E00401674038C068D0712520D74011251FF46
:10017E009007BEEEF0A3EFF07E017F00900096E0B8
:10018E0012520D9000D9E08E048F05FF1200857477
:10019E000AFF1200858D399000E2E075F0DCA4FFB5
:1001AE00AEF0740A8E048F05FF1200859007C4EC22
:1001BE00F0A3EDF09000E4E060139000E4E0F5F0C1
:1001CE00741684FF7E00EF9007CCF0800674649066
:1001DE0007CCF09000C0E0B4020674019000C0F0AD
:1001EE009000ECE0B4010674009000C0F09000C3E3
:1001FE00E0B40B0874E3900085F080499000C3E0F2
:10020E00B419129000D9E0904F0C1251F0E4939073
:10021E000085F080309000C3E0B41E129000D9E04B
:10022E00904F2A1251F0E493900085F080179000C1
:10023E00C3E0B428109000D9E0904F541251F0E46E
:10024E0093900085F09000F6E0B4011790002C74A6
:10025E000FF0A374FFF090002EE4F0A3F074029060
:10026E0000F6F09000F6E0B4034190002EE0FEA3FD
:10027E00E0FF90002CE0FCA3E0FD12526C74101213
:10028E00520D74081251FFEF900082F0EF70067459
:10029E00FF900082F074009000F6F090002DE09038
:1002AE000083F090002CE0900084F0900087E090A6
:1002BE000044F0900044E0240C900045F09000447F
:1002CE00E02418900046F0900044E024249000476B
:1002DE00F0900044E02430900048F0900045E0D3C8
:1002EE00943C400B900045E0C3943C900045F09048
:1002FE000046E0D3943C400B900046E0C3943C9003
:10030E000046F0900047E0D3943C400B900047E04D
:10031E00C3943C900047F0900048E0D3943C400BCF
:10032E00900048E0C3943C900048F090004EE4F0FA
:10033E00900044E0643B6007900044E0B43C2090A1
:10034E000044E0B43B06740290004EF0900044E08E
:10035E00B43C0690004E7401F09000447401F0908D
:10036E00004FE4F0900045E0643B6007900045E0EC
:10037E00B43C20900045E0B43B06740290004FF070
:10038E00900045E0B43C0690004F7401F09000459B
:10039E007401F0900050E4F0900046E0643B60077A
:1003AE00900046E0B43C20900046E0B43B06740258
:1003BE00900050F0900046E0B43C0690005074015E
:1003CE00F09000467401F0900051E4F0900047E088
:1003DE00643B6007900047E0B43C20900047E0B4D7
:1003EE003B067402900051F0900047E0B43C06903A
:1003FE0000517401F09000477401F0900052E4F047
:10040E00900048E0643B6007900048E0B43C2090C8
:10041E000048E0B43B067402900052F0900048E0B1
:10042E00B43C069000527401F09000487401F090B4
:10043E000087E0FE9000EAE02E900054F090005409
:10044E00E0D3943C400B900054E0C3943C90005495
:10045E00F0900054E0B41E06741F900054F090000B
:10046E0054E0B43C069000547401F0900054E064E3
:10047E001D6007900054E0B43206900054E014F072
:10048E00900054E0D3941E400D900054E0C3941E8F
:10049E00900055F0800A900054E0241E900055F014
:1004AE009000CDE0900049F0900049E0640B601799
:1004BE00900049E06417600F900049E064236007E4
:1004CE00900049E0B42F06900049E014F0900049E6
:1004DE00E0640C6017900049E06418600F900049CA
:1004EE00E064246007900049E0B43006900049E0D3
:1004FE0004F0900049E0240C90004AF0900049E08E
:10050E00241890004BF0900049E0242490004CF009
:10051E00900049E0243090004DF090004AE0D394D2
:10052E003C400B90004AE0C3943C90004AF090008F
:10053E004BE0D3943C400B90004BE0C3943C9000B6
:10054E004BF090004CE0D3943C400B90004CE0C339
:10055E00943C90004CF090004DE0D3943C400B90B6
:10056E00004DE0C3943C90004DF022C293C294C261
:10057E0091C292C287C290E5B554EFF5B5E5B55478
:10058E00DFF5B5C296C295C2A0C297C2A2C2A1E5BE
:10059E00B5547FF5B5E5B554BFF5B5E5B554FBF5E6
:1005AE00B5C20D7537469000D0E0700575490280D2
:1005BE000375490390001474FFF0A374DCF09000EF
:1005CE00B1E090001AF8E4F0E8A3F0C213C215C22D
:1005DE0017C219C21B74C8900030F074C890003452
:1005EE00F074C8900038F074C890003CF074C89055
:1005FE000040F0752600752500C208756C00E54BAD
:10060E00B40903754B00753C00900022E4F0A3F092
:10061E00754C1E752800752700C210C211C21290AB
:10062E0007C0E0FEA3E0FF740312520D74011251D5
:10063E00FF9007BEEEF0A3EFF0C203900018E4F0B7
:10064E00A3F0C22122053D2285A74F75A710A2D87F
:10065E00B34002C293A2D9B34002C294A2DAB3400D
:10066E0002C291A2DBB34002C292A2DCB34002C22C
:10067E008775D840854FA722900047E493640660A3
:10068E000280FE74C89007C6F8E4F0E8A3F075B5D2
:10069E000075840175A70075FF8075EF06900053F5
:1006AE00E4F075C91075A70F75A1C775A70075D9A8
:1006BE000075CE0C75A70F75F1FE75F2FF75F30779
:1006CE0075F47875A4BA75A5FF75A60775AE007595
:1006DE00AFFF75D48175D5FF75D6FF75D7FF75A79A
:1006EE000075A20175A14775F80975D80075D90472
:1006FE0075A71075D80075D90475DA0975DB0975FB
:10070E00DC0975DD0975DE0975D84075A70075E63B
:10071E000075E71075BC0175BE0475BD6C75BE071E
:10072E0075BDA075BE0875BD0175BC0075BB18758D
:10073E00BC2075BA0875E88075D11375B50075A71C
:10074E000F75E10575E20075C740C293C294C29160
:10075E00C292C287C290E5B554EFF5B5E5B554DF48
:10076E00F5B5C296C295C2A0C297C2A2C2A1E5B506
:10077E00547FF5B5E5B554BFF5B5E5B554FBF5B504
:10078E00759700759780740A1200757597C0E59776
:10079E005420700280F8758F0275A700D2AF75983D
:1007AE000075A90C75A70F75AB4375ADFB75AC1E27
:1007BE0075A71075C91875CA0075CB0075C8047574
:1007CE00A700758912758E04758C00758A00C2A9F2
:1007DE00D28C758D00758B00D2ABD28E75D94475C7
:1007EE003200753100752E00752D00754600754767
:1007FE0000C29974C8F50975080012329075B500DB
:10080E0074639007C6F8E4F0E8A3F012351C746424
:10081E00F509750800123290C220900070E0B40104
:10082E0008A2B54002D220802E900070E0B40211D2
:10083E0075A70F75F30F75A700A2A34002D22080F3
:10084E0016900070E0B4030F75A70F75F31775A718
:10085E0000A2A44002D220A220B350030209537476
:10086E00089007C6F8E4F0E8A3F01233EB7464F5D1
:10087E000975080012329074099007C6F8E4F0E882
:10088E00A3F01233EB7464F50975080012329074FC
:10089E000A9007C6F8E4F0E8A3F01233EB7464F59F
:1008AE0009750800123290740B9007C6F8E4F0E850
:1008BE00A3F01233EB7464F50975080012329074CC
:1008CE000C9007C6F8E4F0E8A3F01233EB7464F56D
:1008DE0009750800123290740D9007C6F8E4F0E81E
:1008EE00A3F01233EB7464F509750800123290749C
:1008FE000E9007C6F8E4F0E8A3F01233EB7464F53B
:10090E000975080012329074029000CFF0900070BA
:10091E00E0900093F0900070E0B401087400900035
:10092E009BF0801C900070E0B4020874009000DE12
:10093E00F0800D900070E0B4030674009000EBF0B0
:10094E00D21E020A339007C6E4F0A304F01233EB72
:10095E007464F50975080012329074029007C6F897
:10096E00E4F0E8A3F01233EB7464F5097508001295
:10097E00329074039007C6F8E4F0E8A3F01233EB5C
:10098E007464F50975080012329074049007C6F865
:10099E00E4F0E8A3F01233EB7464F5097508001265
:1009AE00329074059007C6F8E4F0E8A3F01233EB2A
:1009BE007464F50975080012329074069007C6F833
:1009CE00E4F0E8A3F01233EB7464F5097508001235
:1009DE00329074079007C6F8E4F0E8A3F01233EBF8
:1009EE007464F50975080012329074019000CFF00E
:1009FE00900070E0900093F0900070E0B4010874E5
:100A0E000090009BF0801C900070E0B4020874000F
:100A1E009000DEF0800D900070E0B403067400903C
:100A2E0000EBF0C21E1236909000D9E07006740AE8
:100A3E009000D9F0900085E0700674E3900085F088
:100A4E00120135E5B54401F5B5740690005FF074FA
:100A5E0001900060F07403900062F07404900063E3
:100A6E00F0741D900064F07404900065F0740390AF
:100A7E000066F0740090006BF0740090006CF074DF
:100A8E000190006DF0740090006EF074FF90006F96
:100A9E00F0743690015DF0743090015EF0742D901C
:100AAE00015FF07432900160F07420900161F07477
:100ABE0035900162F07443900163F0747990016493
:100ACE00F0746C900165F07420900166F0742090C3
:100ADE000167F07420900168F07420900169F07441
:100AEE002090016AF0742090016BF09000F5E09078
:100AFE000082F09000ACE0900083F09000ADE090AA
:100B0E000084F0C213C215C217C219C21B74C8905A
:100B1E000030F074C8900034F074C8900038F0744F
:100B2E00C890003CF074C8900040F0C210C211C2D0
:100B3E0012A2B6B39209A2B3B3920A752600752516
:100B4E0000753746754C1E90007EE4F075271975BA
:100B5E00286490001474FFF0A374DCF0C20D754B82
:100B6E0000C208752A00752900900018E4F0A3F061
:100B7E00743A900786F074FD900787F0756D0090BB
:100B8E00007FE4F0752C00752B0090001CE4F0A3A0
:100B9E00F09000B1E090001AF8E4F0E8A3F09000B5
:100BAE0092E075F032A4FFAEF090002AEEF0A3EFC3
:100BBE00F09007C0E0FEA3E0FF740312520D740123
:100BCE001251FF9007BEEEF0A3EFF0754A0174FAD2
:100BDE0090005BF0C221756C00753C00C20EC20F16
:100BEE00C222C203754D00C204D205C206D207D27C
:100BFE001F74FE900056F074FE900057F07538008A
:100C0E00754400753A00753E32753F0075400074AC
:100C1E003C900059F0743C90005AF07541007542BA
:100C2E0000754300900022E4F0A3F0754500D2B2A7
:100C3E00D2A4D2B0D2B1D2A3D2A7D2A6D2A5D2B7C5
:100C4E00900092E0D394FA400674FA900092F07EEF
:100C5E00017F00900084E012520D900083E02FFF80
:100C6E0050010E90002CEEF0A3EFF0EFD394FFEEB8
:100C7E00940F400790002CE4F0A3F0900082E070F7
:100C8E000674FF900082F09000CFE0D394024006ED
:100C9E0074019000CFF09000D0E07005754902808D
:100CAE00037549039000D1E0D3940140067400907F
:100CBE0000D1F09000D7E0C3940A5006740A900059
:100CCE00D7F09000E1E0700674019000E1F0900022
:100CDE00E1E0B4FF0674FE9000E1F09000E8E0D38E
:100CEE0094FE400674FE9000E8F074019000EEF061
:100CFE0074019000EFF074009000F1F07400900019
:100D0E00F6F0D29CD2EC75CF01A298B3500302112B
:100D1E000AC298E54764046006E59964FF600280A4
:100D2E001EE547600874E6254790005BF0754700A6
:100D3E00E546600874F0254690005BF0754600E5C8
:100D4E00476003020DEF754700E599B4FF03754642
:100D5E0001E599B4FE03754602E599B4FD037546A7
:100D6E0003E599B4FC03754604E599B4FA03754698
:100D7E0005E599B4FB03754701E599B4F903754789
:100D8E0004E599D394E54007E599C394F0400280B9
:100D9E00168599487547027E017F00E548C394E6A3
:100DAE0012520D8E2F8F30753200753100E599D3AA
:100DBE0094C74007E599C394E64002801F85994881
:100DCE0075470374E5C39548F530752F00AE2FAF08
:100DDE0030904FA51200647831125252D2990211FE
:100DEE000AE547B401028003020ECDE532453170AB
:100DFE0003120579AE31AF32900086125234E59966
:100E0E00F07831125274AE31AF32EFB40106EEB457
:100E1E0007028003020ECD900786E0B43C028003E9
:100E2E00020EB7C29C120135900082E09000F5F0E0
:100E3E00900083E09000ACF0900084E09000ADF064
:100E4E00A21E4032755001E550D394075026E5504E
:100E5E009007C6F8E4F0E8A3F074AA900053F012DD
:100E6E0032BC7464F5097508001232907850740122
:100E7E0026F650D38030755008E550D3940E502688
:100E8E00E5509007C6F8E4F0E8A3F074AA9000537A
:100E9E00F01232BC7464F509750800123290785065
:100EAE00740126F650D312369074C89007C6F8E433
:100EBE00F0E8A3F0D29C7547007546007599FBE5E6
:100ECE0047B402028003020F61E532453170068598
:100EDE00992E752D00AE31AF3274016F4E701BAC72
:100EEE002DAD2EAA2FAB30ED2BFBEC3AFA8A068BEA
:100EFE0007900086125234E599F07831125274AE92
:100F0E0031AF3274026F4E704AAC2DAD2E740D6D32
:100F1E004C702774639007C6F8E4F0E8A3F074AB46
:100F2E00900053F0900093E0900070F01235F5743D
:100F3E00C89007C6F8E4F0E8A3F0AE2DAF2E7456B5
:100F4E006F4E700312057912013585489975470069
:100F5E00754600E547B4033FAE31AF3290008612BE
:100F6E005234E599F07831125274AE31AF32AC2F63
:100F7E00AD308F028E038C068D07904FE112006408
:100F8E00E493F9740193FEEAD39EEB9940098548E8
:100F9E0099754700754600E547B4040280030211B7
:100FAE000AE53245317003120579AE31AF32900049
:100FBE0086125234E599F07831125274AE31AF3256
:100FCE00EFB40006EEB40102800302110A9000692C
:100FDE00E075F002A4FDACF08D50ED90008612523B
:100FEE0049EDFAE0FBEA900089125249EBFAE0FB78
:100FFE00EA2BFA900069E0B5020280030210FB0DA5
:10100E00ED900086125249E550FDE0FAED90008A0F
:10101E00125249EAFDE0FAEDC39AFD900069E0B57F
:10102E00050280030210FBE550900088125249E53C
:10103E0050FDE0FAED90008B125249EAFDE0FAED18
:10104E002AFD900069E0B5050280030210FBE55011
:10105E0090008C125249FDE0FAED900069E0F40424
:10106E002A900070F0E55090008D125249FDE0FA82
:10107E00ED900069E0F4042A900071F0E5509000C4
:10108E008E125249FDE0FAED900069E0F4042A90C8
:10109E000072F0E55090008F125249FDE0FAED908B
:1010AE000069E0F4042A9007C6F8E4F0E8A3F074AF
:1010BE00AB900053F01235F57464F5097508001203
:1010CE0032909007C612521B1235F57464F50975ED
:1010DE0008001232909007C612521B1235F5759900
:1010EE00F97464F50975080012329080FE7599FF47
:1010FE007464F50975080012329080FEE5466006AC
:10110E00A299B3B3400302126BC299E546B4011F14
:10111E00AE31AF3290005F125234E0F59978311251
:10112E005274AE31AF3274116F4E7003754600E5D6
:10113E0046B40203854A99E546B4031DAE31AF327B
:10114E00900086125234E0F599EFB40107EEB40721
:10115E00037546007831125274E546B404028003DA
:10116E0002124AE53245317003852699AE31AF320F
:10117E0074016F4E7003853899AE31AF3274026FC1
:10118E004E7003853A99AE31AF3274036F4E7003D1
:10119E00853E99AE31AF3274046F4E70038540991F
:1011AE00AE31AF3274056F4E7003854199AE31AFDB
:1011BE003274066F4E7003854299AE31AF327407AA
:1011CE006F4E7003854399AE31AF3274086F4E7017
:1011DE0006900023E0F599AE31AF3274096F4E7070
:1011EE000690005BE0F599AE31AF32740A6F4E7027
:1011FE0003854499AE31AF32740B6F4E7003853F49
:10120E0099AE31AF32740C6F4E7003854599AE3185
:10121E00AF32740D6F4E700590005BE4F0AE31AFDF
:10122E0032740D6F4E70037599FC7831125274AE94
:10123E0031AF32740E6F4E7003754600E546B4053D
:10124E001CAE31AF32904E3A125234E493F599748B
:10125E00E66F4E70037546007831125274E547649E
:10126E00016005E547B40403020D14C28E7E107FA3
:10127E0000E53D12520DE58D75F010A4FDACF0EFBA
:10128E002DFDEE3CFCE58B75F01084FF7E00ED2FFE
:10129E00FFEC3EFE8E278F28D28E9000B3E0605674
:1012AE0090002412521B900024E0FCA3E0FD90005D
:1012BE0026E0FAA3E0FBEDB5033CECB50238B21D17
:1012CE00A208B34013A21DB34008E5B54404F5B51A
:1012DE008006E5B554FBF5B5900026E0FEA3E0FFD1
:1012EE00900028E0FCA3E0FDEF2DFDEE3CFC90000D
:1012FE0026ECF0A3EDF09000ECE060030213A49056
:10130E0000C0E060099000C0E0C394034002806317
:10131E00124B90A208B3500990007EE0C394464051
:10132E000280069000AAE0F56BE56B75F005A4FF50
:10133E00AEF09007C8EEF0A3EFF0900097E0C395E3
:10134E003A4007E538C3953950079007C8E4F0A333
:10135E00F0AE58AF599007C8E0FCA3E0FDEFD39D67
:10136E00EE9C4004C2A1800B90007EE0C3946450BA
:10137E0002D2A19000C0E0B4031C124C8CAE58AF48
:10138E00599007C8E0FCA3E0FDEFD39DEE9C40040E
:10139E00D2A18002C2A1A2B6300901B35003021835
:1013AE00FEA2B6300901B350030218FEA2B6300BEE
:1013BE0001B35003021817754A009000B3E0701382
:1013CE00A20BB34008E5B554FBF5B58006E5B54470
:1013DE0004F5B50537A20DB3B35013AE27AF289061
:1013EE000014E0FCA3E0FDEDC39FEC9E400302144D
:1013FE00DAE549B40330E537B43B05754901801F82
:10140E00A221B3401AE537C3943B500690005B749B
:10141E0001F0E537D3943B4006740290005BF07503
:10142E003701D2218044E549B4020675490175376A
:10143E003BE537B43B05753701802F90005BE070BC
:10144E001AE537C3943B500690005B7401F0E53704
:10145E00D3943B4006740290005BF09000D0E0B451
:10146E0002051205798003753701AE29AF2AAC2724
:10147E00AD28EF2DFDEE3CFC74028C068D0712514B
:10148E00FF8E298F2A9000B3E0603F900024E0FC8D
:10149E00A3E0FD9000B3E0FF12008574018C068D71
:1014AE00071251FF900028EEF0A3EFF0900028E015
:1014BE00F8A3E0900026C8F0A3C8F0900024E4F052
:1014CE00A3F0C21DE5B554FBF5B5802BAE29AF2AAE
:1014DE00AC27AD28EF2DFDEE3CFC74018C068D077C
:1014EE001251FF8E298F2AAC27AD28EDD394B8EC7C
:1014FE00940B4003120579E537B43B10740390004A
:10150E005BF09000D0E0B40203120579AE2BAF2C45
:10151E00AC27AD28EF2DFDEE3CFC8C2B8D2CAE2791
:10152E00AF28EFD39DEE9C401190001CE0FAA3E093
:10153E00FBEBC394E8EA94034002800690001C1271
:10154E00521B900018E0FEA3E0FFAC27AD28EF2D54
:10155E00FDEE3CFC900018ECF0A3EDF09000D0E016
:10156E00B40218AE27AF28740512520D7401125131
:10157E00FF900014EEF0A3EFF08011AE27AF2874A9
:10158E000212520D900014EEF0A3EFF0C28E758D84
:10159E0000758B00753D00752801752700D28EE50C
:1015AE0037240E75F00F84AFF07E00EF4E707590FD
:1015BE000018E0F8A3E0900016C8F0A3C8F0900061
:1015CE0016E0FEA3E0FFEF4E600B7C817D5A1251B8
:1015DE000F8E258F26900018E4F0A3F0AE25AF26CF
:1015EE007428BE00039F5010E53C2FFF50010E746F
:1015FE00011251FF8E258F2685263C9000D7E0A83C
:10160E0025B8000DD395264008E526900058F080A9
:10161E00099000D7E014900058F0E5496006752651
:10162E0000752500E537640B6005E537B429099090
:10163E0000C0E060031248D2900054E065376007A6
:10164E00900055E0B53703754B00A20E50030217FC
:10165E003890008CE0B4015AE54075F00584FF7EA9
:10166E0000900586125234E0F534753300AE33AF78
:10167E003490008AE012520D74648E048F05FF12AE
:10168E00008574C18C068D0712520D8E358F3690E3
:10169E00001AE0FEA3E0FFAC33AD34120003746415
:1016AE008E048F05FF12008590001AECF0A3EDF06A
:1016BE00800F90008AE075F0C1A4FFAEF08E358FDA
:1016CE0036E53AC394CC506075A71085F95085FA6B
:1016DE00517E017F00E55112520DE5502FFF500152
:1016EE000E8E338F34AC35AD36EF2DFDEE3CFC8CCB
:1016FE00358D36D293D294D291D292D287E536F5E9
:10170E00FBE535F5FCE536F5E9E535F5EAE536F5C3
:10171E00EBE535F5ECE536F5EDE535F5EEE536F5CB
:10172E00FDE535F5FE75A700D20EE549B40106E5D7
:10173E003764116002800F754C0190005E7401F0E9
:10174E00E5B54401F5B5E54960030218129000D3E2
:10175E00E0600D9000DAE0A825B80006952640025C
:10176E00804A9000D3E0B4022F900044E0653760C9
:10177E001F900045E065376017900046E0653760C2
:10178E000F900047E065376007900048E0B53703DB
:10179E00754C03754500800CC20075450090002203
:1017AE00E4F0A3F0740990005BF08058900044E0E0
:1017BE00B5370B754C0190005E7401F080469000B9
:1017CE0045E0B5370B754C01740290005EF0803425
:1017DE00900046E0B5370B754C01740390005EF037
:1017EE008022900047E0B5370B754C0174049000D1
:1017FE005EF08010900048E0B53709754C01740515
:10180E0090005EF0A20BB39209A20BB330B601B3F7
:10181E0050030218FE754A019000B3E07013A20B3C
:10182E00B34008E5B54404F5B58006E5B554FBF5BF
:10183E00B5A20B9209E537D3944A4012D20DE53783
:10184E00D394854009740390005BF0753746900081
:10185E00DBE0B40107E543C3941440028003120594
:10186E0079744690007EF0A204300501B35017A2A1
:10187E0004B34008E5B54408F5B58006E5B554F760
:10188E00F5B5A2049205A206300701B35017A206C1
:10189E00B34008E5B54402F5B58006E5B554FDF54F
:1018AE00B5A2069207E543C394415009740E900009
:1018BE005BF0120579900065E0FE900061E004C3D4
:1018CE009E4009900061E0D39406400974FB90009D
:1018DE005BF012057990006AE0601590006AE0FEF8
:1018EE00900064E06E600974FE90005BF012057962
:1018FE00A210B3B35008900049E0653760028060D3
:10190E00A202B35006A200B3B34002804D9000EC89
:10191E00E0600BA203B34004D2A18002C2A175A75E
:10192E001085F95085FA517E017F00E55112520D56
:10193E00E5502FFF50010E8E338F34900020E0FCC7
:10194E00A3E0FDEF2DFDEE3CFC8C358D36E536F536
:10195E00FBE535F5FC75A700D293C210D211D21259
:10196E00A211B3B3500890004AE065376002806060
:10197E00A202B35006A200B3B34002804D9000EC19
:10198E00E0600BA203B34004D2A18002C2A175A7EE
:10199E001085F95085FA517E017F00E55112520DE6
:1019AE00E5502FFF50010E8E338F34900020E0FC57
:1019BE00A3E0FDEF2DFDEE3CFC8C358D36E536F5C6
:1019CE00E9E535F5EA75A700D294D210C211D2120C
:1019DE00A212B3B3500890004BE0653760028060EE
:1019EE00A202B35006A200B3B34002804D9000ECA9
:1019FE00E0600BA203B34004D2A18002C2A175A77E
:101A0E001085F95085FA517E017F00E55112520D75
:101A1E00E5502FFF50010E8E338F34900020E0FCE6
:101A2E00A3E0FDEF2DFDEE3CFC8C358D36E536F555
:101A3E00EBE535F5EC75A700D291D210D211C2129A
:101A4E00A210B3B3500890004CE06537600280607E
:101A5E00A202B35006A200B3B34002804D9000EC38
:101A6E00E0600BA203B34004D2A18002C2A175A70D
:101A7E001085F95085FA517E017F00E55112520D05
:101A8E00E5502FFF50010E8E338F34900020E0FC76
:101A9E00A3E0FDEF2DFDEE3CFC8C358D36E536F5E5
:101AAE00EDE535F5EE75A700D292C210D211D21225
:101ABE00A211B3B3500890004DE06537600280600C
:101ACE00A202B35006A200B3B34002804D9000ECC8
:101ADE00E0600BA203B34004D2A18002C2A175A79D
:101AEE001085F95085FA517E017F00E55112520D95
:101AFE00E5502FFF50010E8E338F34900020E0FC06
:101B0E00A3E0FDEF2DFDEE3CFC8C358D36E536F574
:101B1E00FDE535F5FE75A700D287D210C211D2129F
:101B2E00E54CB40818124201A210B35005A211B32D
:101B3E0040028006D210D211D212754C1EE54CB462
:101B4E000706123FB9754C08E54CB4063D90001AD5
:101B5E00E0FEA3E0FFEF4E6006A208B3B3400280A2
:101B6E0023AE52AF5390001AE0FCA3E0FDEF2DFD23
:101B7E00EE3CFC8C528D53E537D3940A5006900000
:101B8E001A120039123D8B754C07E54CB40506123E
:101B9E003BEB754C06E54CB404329000C1E090323C
:101BAE0072F828287312387F801212387F800D1237
:0C1BBE003A2D8008123ADF8003123ADF53
:0F327200021BB3021BB8021BBD021BC2021BC70B
:101BCA009000A3E060051249BB8002C204754C056F
:101BDA00E54CB403028003021CC49000A6E0600531
:101BEA00124AAB8002C2069000C1E0D39402403F81
:101BFA00900095E02403A825B80004952650099082
:101C0A000097E0D3953A50028008D20274089000F7
:101C1A005BF0900095E0A825B80005D39526500BF7
:101C2A00900097E02403C3953A5002C2028039908B
:101C3A000095E02403A825B8000495265007E53846
:101C4A00C3953940028008D202740890005BF09074
:101C5A000095E0A825B80005D395265009E5392452
:101C6A000FC395385002C2029000DBE07007E543CB
:101C7A00C3941440028002D202A2024005754C04A9
:101C8A00800A754C1E900022E4F0A3F0A208B3402B
:101C9A0029E54075F00584FF7E00900586125234CE
:101CAA00E0C394695005124907800F9007C0E0F815
:101CBA00A3E09007BEC8F0A3C8F0E54CB40A0280BE
:101CCA0003021D86900032E0C394465008C29674FF
:101CDA0046900032F090004EE0B4011DE55A240609
:101CEA00F55A9007C2E0FEA3E0FF74062FFF5001E9
:101CFA000E9007C2EEF0A3EFF090004EE0B4021D82
:101D0A00E55A240CF55A9007C2E0FEA3E0FF740CD2
:101D1A002FFF50010E9007C2EEF0A3EFF0855A3460
:101D2A00753300900044E0F55012009EE5369000AD
:101D3A0032F090000AE533F0A3E534F0E550900064
:101D4A0033F0C2149007C2E0F533A3E0F5349000F3
:101D5A0044E0F55012009EE536900030F090000005
:101D6A00E533F0A3E534F0E550900031F0C213E515
:101D7A0049B40105754C0B8003754C03900030E0A3
:101D8A00B537028003021E25A2134072900000E0BC
:101D9A00FEA3E0FFEF4E6021AE29AF2A900000E0DB
:101DAA00FCA3E0FD12000374068E048F05FF1200E7
:101DBA0085900000ECF0A3EDF0900031E0601A90FD
:101DCA000000E0FEA3E0FFAC29AD2AEF2DFDEE3CBA
:101DDA00FC900000ECF0A3EDF0900031E0D3940108
:101DEA00401A900000E0FEA3E0FFAC29AD2AEF2DD7
:101DFA00FDEE3CFC900000ECF0A3EDF0D213AE2710
:101E0A00AF28900000E0FCA3E0FDEFC39DEE9C40EC
:101E1A000AD296C21374C8900030F0A213B3B3501A
:101E2A0007900030E0B53702800AD29674C8900055
:101E3A0030F0C213900032E0B537028003021EDD93
:101E4A00A214407290000AE0FEA3E0FFEF4E602168
:101E5A00AE29AF2A90000AE0FCA3E0FD1200037449
:101E6A00068E048F05FF12008590000AECF0A3EDA0
:101E7A00F0900033E0601A90000AE0FEA3E0FFACA5
:101E8A0029AD2AEF2DFDEE3CFC90000AECF0A3ED03
:101E9A00F0900033E0D39401401A90000AE0FEA3C8
:101EAA00E0FFAC29AD2AEF2DFDEE3CFC90000AECD8
:101EBA00F0A3EDF0D214AE27AF2890000AE0FCA3FD
:101ECA00E0FDEFC39DEE9C400AC296744690003234
:101EDA00F0C214A214B3B35007900032E0B537022F
:101EEA00800AC2967446900032F0C214E54CB40BD4
:101EFA00028003021FB8900036E0C394465008C21D
:101F0A00967446900036F090004FE0B4011DE55AF1
:101F1A002406F55A9007C2E0FEA3E0FF74062FFFDD
:101F2A0050010E9007C2EEF0A3EFF090004FE0B41C
:101F3A00021DE55A240CF55A9007C2E0FEA3E0FF01
:101F4A00740C2FFF50010E9007C2EEF0A3EFF0853C
:101F5A005A34753300900045E0F55012009EE5367C
:101F6A00900036F090000CE533F0A3E534F0E5502C
:101F7A00900037F0C2169007C2E0F533A3E0F534BB
:101F8A00900045E0F55012009EE536900034F0903E
:101F9A000002E533F0A3E534F0E550900035F0C2D5
:101FAA0015E549B40105754C0C8003754C03900086
:101FBA0034E0B537028003022057A2154072900020
:101FCA0002E0FEA3E0FFEF4E6021AE29AF2A9000A7
:101FDA0002E0FCA3E0FD12000374068E048F05FFE5
:101FEA00120085900002ECF0A3EDF0900035E0605D
:101FFA001A900002E0FEA3E0FFAC29AD2AEF2DFD06
:10200A00EE3CFC900002ECF0A3EDF0900035E0D33A
:10201A009401401A900002E0FEA3E0FFAC29AD2A29
:10202A00EF2DFDEE3CFC900002ECF0A3EDF0D21592
:10203A00AE27AF28900002E0FCA3E0FDEFC39DEEBF
:10204A009C400AD296C21574C8900034F0A215B307
:10205A00B35007900034E0B53702800AD29674C8AC
:10206A00900034F0C215900036E0B53702800302C2
:10207A00210FA216407290000CE0FEA3E0FFEF4E83
:10208A006021AE29AF2A90000CE0FCA3E0FD12000B
:10209A000374068E048F05FF12008590000CECF085
:1020AA00A3EDF0900037E0601A90000CE0FEA3E088
:1020BA00FFAC29AD2AEF2DFDEE3CFC90000CECF0B4
:1020CA00A3EDF0900037E0D39401401A90000CE0A1
:1020DA00FEA3E0FFAC29AD2AEF2DFDEE3CFC9000FB
:1020EA000CECF0A3EDF0D216AE27AF2890000CE06E
:1020FA00FCA3E0FDEFC39DEE9C400AC29674469095
:10210A000036F0C216A216B3B35007900036E0B5F7
:10211A003702800AC2967446900036F0C216E54C21
:10212A00B40C0280030221EA90003AE0C3944650BC
:10213A0008C296744690003AF0900050E0B4011D2F
:10214A00E55A2406F55A9007C2E0FEA3E0FF74069A
:10215A002FFF50010E9007C2EEF0A3EFF09000504F
:10216A00E0B4021DE55A240CF55A9007C2E0FEA31A
:10217A00E0FF740C2FFF50010E9007C2EEF0A3EFA0
:10218A00F0855A34753300900046E0F55012009EEF
:10219A00E53690003AF090000EE533F0A3E534F00E
:1021AA00E55090003BF0C2189007C2E0F533A3E077
:1021BA00F534900046E0F55012009EE5369000385E
:1021CA00F0900004E533F0A3E534F0E550900039CF
:1021DA00F0C217E549B40105754C0D8003754C032F
:1021EA00900038E0B537028003022289A2174072B4
:1021FA00900004E0FEA3E0FFEF4E6021AE29AF2A73
:10220A00900004E0FCA3E0FD12000374068E048F24
:10221A0005FF120085900004ECF0A3EDF090003960
:10222A00E0601A900004E0FEA3E0FFAC29AD2AEFBB
:10223A002DFDEE3CFC900004ECF0A3EDF09000398B
:10224A00E0D39401401A900004E0FEA3E0FFAC2919
:10225A00AD2AEF2DFDEE3CFC900004ECF0A3EDF06E
:10226A00D217AE27AF28900004E0FCA3E0FDEFC32D
:10227A009DEE9C400AD296C21774C8900038F0A20C
:10228A0017B3B35007900038E0B53702800AD296E8
:10229A0074C8900038F0C21790003AE0B53702804F
:1022AA0003022341A218407290000EE0FEA3E0FF51
:1022BA00EF4E6021AE29AF2A90000EE0FCA3E0FDAC
:1022CA0012000374068E048F05FF12008590000E1B
:1022DA00ECF0A3EDF090003BE0601A90000EE0FEF7
:1022EA00A3E0FFAC29AD2AEF2DFDEE3CFC90000ED9
:1022FA00ECF0A3EDF090003BE0D39401401A90007B
:10230A000EE0FEA3E0FFAC29AD2AEF2DFDEE3CFC6A
:10231A0090000EECF0A3EDF0D218AE27AF28900093
:10232A000EE0FCA3E0FDEFC39DEE9C400AC296744A
:10233A004690003AF0C218A218B3B3500790003A78
:10234A00E0B53702800AC296744690003AF0C21885
:10235A00E54CB40D02800302241C90003EE0C394B5
:10236A00465008C296744690003EF0900051E0B480
:10237A00011DE55A2406F55A9007C2E0FEA3E0FFC4
:10238A0074062FFF50010E9007C2EEF0A3EFF090F3
:10239A000051E0B4021DE55A240CF55A9007C2E038
:1023AA00FEA3E0FF740C2FFF50010E9007C2EEF05F
:1023BA00A3EFF0855A34753300900047E0F55012C8
:1023CA00009EE53690003EF0900010E533F0A3E55C
:1023DA0034F0E55090003FF0C21A9007C2E0F5339E
:1023EA00A3E0F534900047E0F55012009EE53690E0
:1023FA00003CF0900006E533F0A3E534F0E5509098
:10240A00003DF0C219E549B40105754C0E8003750B
:10241A004C0390003CE0B5370280030224BBA219AA
:10242A004072900006E0FEA3E0FFEF4E6021AE2965
:10243A00AF2A900006E0FCA3E0FD12000374068EAA
:10244A00048F05FF120085900006ECF0A3EDF090D2
:10245A00003DE0601A900006E0FEA3E0FFAC29AD63
:10246A002AEF2DFDEE3CFC900006ECF0A3EDF09077
:10247A00003DE0D39401401A900006E0FEA3E0FF7D
:10248A00AC29AD2AEF2DFDEE3CFC900006ECF0A342
:10249A00EDF0D219AE27AF28900006E0FCA3E0FDCC
:1024AA00EFC39DEE9C400AD296C21974C890003CB4
:1024BA00F0A219B3B3500790003CE0B53702800A86
:1024CA00D29674C890003CF0C21990003EE0B5372D
:1024DA00028003022573A21A4072900010E0FEA344
:1024EA00E0FFEF4E6021AE29AF2A900010E0FCA376
:1024FA00E0FD12000374068E048F05FF120085901A
:10250A000010ECF0A3EDF090003FE0601A9000108C
:10251A00E0FEA3E0FFAC29AD2AEF2DFDEE3CFC90D6
:10252A000010ECF0A3EDF090003FE0D39401401AC4
:10253A00900010E0FEA3E0FFAC29AD2AEF2DFDEEDE
:10254A003CFC900010ECF0A3EDF0D21AAE27AF28B5
:10255A00900010E0FCA3E0FDEFC39DEE9C400AC290
:10256A0096744690003EF0C21AA21AB3B35007906E
:10257A00003EE0B53702800AC296744690003EF0EB
:10258A00C21AE54CB40E02800302266A900042E0A9
:10259A00C394465008C2967446900042F090005286
:1025AA00E0B4011DE55A2406F55A9007C2E0FEA3DD
:1025BA00E0FF74062FFF50010E9007C2EEF0A3EF62
:1025CA00F0900052E0B4021DE55A240CF55A900727
:1025DA00C2E0FEA3E0FF740C2FFF50010E9007C269
:1025EA00EEF0A3EFF0855A34753300900048E0F519
:1025FA005012009EE536900042F0900012E533F04A
:10260A00A3E534F0E550900043F0C21C9007C2E005
:10261A00F533A3E0F534900048E0F55012009EE54A
:10262A0036900040F0900008E533F0A3E534F0E579
:10263A0050900041F0C21BE549B40121754900746C
:10264A00C8900030F074C8900034F074C890003814
:10265A00F074C890003CF074C8900040F0754C03C8
:10266A00900040E0B537028003022709A21B40729E
:10267A00900008E0FEA3E0FFEF4E6021AE29AF2AEA
:10268A00900008E0FCA3E0FD12000374068E048F9C
:10269A0005FF120085900008ECF0A3EDF0900041D0
:1026AA00E0601A900008E0FEA3E0FFAC29AD2AEF33
:1026BA002DFDEE3CFC900008ECF0A3EDF0900041FB
:1026CA00E0D39401401A900008E0FEA3E0FFAC2991
:1026DA00AD2AEF2DFDEE3CFC900008ECF0A3EDF0E6
:1026EA00D21BAE27AF28900008E0FCA3E0FDEFC3A1
:1026FA009DEE9C400AD296C21B74C8900040F0A27C
:10270A001BB3B35007900040E0B53702800AD29657
:10271A0074C8900040F0C21B900042E0B5370280B6
:10272A00030227C1A21C4072900012E0FEA3E0FF40
:10273A00EF4E6021AE29AF2A900012E0FCA3E0FD23
:10274A0012000374068E048F05FF12008590001292
:10275A00ECF0A3EDF0900043E0601A900012E0FE66
:10276A00A3E0FFAC29AD2AEF2DFDEE3CFC90001250
:10277A00ECF0A3EDF0900043E0D39401401A9000EE
:10278A0012E0FEA3E0FFAC29AD2AEF2DFDEE3CFCE2
:10279A00900012ECF0A3EDF0D21CAE27AF28900007
:1027AA0012E0FCA3E0FDEFC39DEE9C400AC29674C2
:1027BA0046900042F0C21CA21CB3B35007900042DC
:1027CA00E0B53702800AC2967446900042F0C21CF5
:1027DA00E54CB40202800302289E12466A1247811F
:1027EA009007BEE0FEA3E0FF740A12520D90001695
:1027FA00E0FCA3E0FD74098F02FF1200858D078CAF
:10280A00038E048A058B0612510F9007C2EEF0A3BD
:10281A00EFF09000DCE0B401087430BE00059F4080
:10282A0002800D74309007C2F8E4F0E8A3F0801B30
:10283A009007C2E0FEA3E0FF74F0BE00039F500BB6
:10284A0074F09007C2F8E4F0E8A3F09007C2E0FE43
:10285A00A3E0FFE55A2FFF50010E9007C2EEF0A346
:10286A00EFF090005EE0B40103754C0A90005EE060
:10287A00B40203754C0B90005EE0B40303754C0C74
:10288A0090005EE0B40403754C0D90005EE0B40560
:10289A0003754C0EE54CB401259000F3E0903281AB
:1028AA00F82828731244088012124408800D124432
:0B28BA0092800812453E800312453E4C
:0F3281000228AE0228B30228B80228BD0228C2D4
:1028C500754C02E54BC394094003023003A2EDB3F6
:1028D5005003023003C2EDE54B6003022A779000F6
:1028E5008FE07003022A669000C5E0B40102800300
:1028F5000229C6900054E0B5370280030229C37E41
:10290500017F00E5BE12520DE5BD2FFF50010E8E71
:10291500338F3490008FE0B40118741012520D906B
:102925000085E08E048F05FF120085ED900056F0BE
:10293500802CAE33AF34741012520D900085E08EAA
:10294500048F05FF120085900056E02DFD50010C07
:1029550074018C068D071251FFEF900056F0E54487
:1029650060089000EBE06402600280219000EDE0D9
:10297500B4011A900056E075F0E7A4FFAEF0E54407
:102985008E048F05FF120085ED900056F0900056DD
:10299500E0FE900057E0D39E4004D21F8002B21F94
:1029A500900056E0900057F09000C1E06401600689
:1029B500A21FB3B340028006900056E0F538022A04
:1029C50064D21F7E017F00E5BE12520DE5BD2FFFCB
:1029D50050010E8E338F3490008FE0B401187410BF
:1029E50012520D900085E08E048F05FF120085EDD3
:1029F500900056F0802CAE33AF34741012520D9007
:102A05000085E08E048F05FF120085900056E02DAD
:102A1500FD50010C74018C068D071251FFEF9000DB
:102A250056F0E54460089000EBE064026002802106
:102A35009000EDE0B4011A900056E075F0E7A4FFB0
:102A4500AEF0E5448E048F05FF120085ED9000562B
:102A5500F09000C1E064016006900056E0F5388012
:102A65000375380090008BE07005754B0180037588
:102A7500BB18E54BB401028003022C1990008BE0D2
:102A85007003022C087E017F00E5BE12520DE5BDE4
:102A95002FFF50010E8E338F349000D1E0B4010F1B
:102AA5007E0F7FFFAC33AD3412526C8E338F349072
:102AB50000F6E0B40245AE33AF3490002CE0FCA341
:102AC500E0FDEDD39FEC9E400A90002CE533F0A38A
:102AD500E534F0AE33AF3490002EE0FCA3E0FDEF1B
:102AE500D39DEE9C400A90002EE533F0A3E534F02B
:102AF500AE33AF3474041251FF8F3A9000F6E07094
:102B05004CAE33AF3490002CE0FCA3E0FDEFD39D39
:102B1500EE9C400912526C8E338F3480067534005A
:102B2500753300AE33AF34741012520D900082E04D
:102B35008E048F05FF1200858C338D347400D39D70
:102B450074019C400585343A8003753AFF9000C1B5
:102B5500E0B401028003022C06A208B3B3500E9024
:102B65000095E0A825B80005D395265003022BFB58
:102B7500900096E075F019A4FFAEF09000D9E08EB4
:102B8500048F05FF1200859000D2E0853AF0A4FF7E
:102B9500AEF074648D028C038E048F05FF120085E0
:102BA500EA2DFDEB3CFC8C338D34E544600F900041
:102BB500EBE0B402089000EDE0640160028017AE1E
:102BC50033AF3474E712520DE5448E048F05FF12BE
:102BD50000858C338D34900056E0A833B8000AD3B5
:102BE50095344005853438800BA21FB3400690000C
:102BF50056E0F538800BA21FB34006900056E0F56D
:102C0500388003753A0090008EE07005754B0280A0
:102C15000375BB19E54BB402028003022CD4900066
:102C25008EE07003022CC3E537D3941E4003022CBB
:102C3500C190002AE0FEA3E0FFE53E125264900039
:102C45002AEEF0A3EFF07E017F00E5BE12520DE5FE
:102C5500BD2FFF50010E8E338F349000FBE07013B3
:102C6500740A12520D74518E048F05FF1200858D62
:102C75003E8019AE33AF34740A12520D8F048E059F
:102C85007E017F95CDCCCD12510F8F3EE53ED3947D
:102C9500644003753E6490002AE0FEA3E0FFE53E34
:102CA5002FFF50010E90002AEEF0A3EFF090009256
:102CB500E0048E048F05FF1200858D3E8003753E6E
:102CC500329000DEE07005754B03800375BB13E59C
:102CD5004BB4035E9000DEE060477E017F00E5BEF9
:102CE50012520DE5BD2FFF50010E8E338F34740443
:102CF5001251FF8F3F9000E0E0853FF0A4FDACF05E
:102D05007464FF1200858D3F9000DFE0853FF0A4DD
:102D1500FFAEF074FF8E048F05FF1200858D4E8087
:102D250003753F0090008CE07005754B04800375BA
:102D3500BB17E54BB404028003022DD590008CE04F
:102D4500B4017C7E017F00E5BE12520DE5BD2FFF6B
:102D550050010E74041251FF8E338F34900059E0E8
:102D65006012900059E01490501D93A833B80006E6
:102D7500953440028006900059E014F0900059E027
:102D8500C394775013900059E00490501D93A833D5
:102D9500B80005D3953450028006900059E004F040
:102DA500900059E0FE9000B2E08E0088F0A4FFAEDE
:102DB500F074648E048F05FF1200858D40800375C5
:102DC500400090008DE07005754B05800375BB16BE
:102DD500E54BB405028003022E6890008DE0B40136
:102DE5007C7E017F00E5BE12520DE5BD2FFF50012F
:102DF5000E74041251FF8E338F3490005AE0601226
:102E050090005AE01490509693A833B80006953474
:102E15004002800690005AE014F090005AE0C394F6
:102E250077501390005AE00490509693A833B80059
:102E350005D395345002800690005AE004F09000C6
:102E45005AE0FE9000B8E08E0088F0A4FFAEF07462
:102E5500648E048F05FF1200858D41800375410046
:102E650075BB1FE54BB406337E017F00E5BE1252EC
:102E75000DE5BD2FFF50010E8E338F3474091252AC
:102E85000D74E68E048F05FF1200858D4390009426
:102E9500E07005754B07800375BB15E54BB407025C
:102EA5008003022FAA900094E07003022F997E01FF
:102EB5007F00E5BE12520DE5BD2FFF50010E8E338A
:102EC5008F3474041251FF8F42900094E0B40115C1
:102ED5009000E8E08542F0A4FFAEF074071251FFC0
:102EE500EF9007CBF0900094E0B402159000E8E075
:102EF5008542F0A4FFAEF074071251FFEF9007CAA8
:102F0500F0900094E0B403028003022F979000D55F
:102F1500E0701CE542C3940A5002D201E542D39405
:102F2500644002C2019000B4E0900080F08063909C
:102F350000B4E070349000E8E08542F0A4FFAEF004
:102F450074FF8E048F05FF120085ED900080F0AEB2
:102F550025AF26741EBE0006D39F4002D201E53A76
:102F6500D394E54002C2018029E542C3940A500D7D
:102F7500AE25AF26741EBE0004D39F50028002D238
:102F850001E53AD394E54002C2019000B4E0900017
:102F950080F080037542009000EBE07005754B08EA
:102FA500800375BB14E54BB408509000EBE0603925
:102FB5007E017F00E5BE12520DE5BD2FFF50010ECB
:102FC5008E338F34EFD39421EE940E40057544FF74
:102FD5008015AE33AF34741012520D74E38E048F26
:102FE50005FF1200858D44800375440090008FE035
:102FF500600575BB1A800375BB18054BD2ECAE276F
:10300500AF28EFD39428EE9423500302326FC20DFC
:103015007537469000D0E070057549028003754903
:1030250003C293C294C291C292C287C290E5B554BD
:10303500EFF5B5E5B554DFF5B5C296C295C2A0C2A8
:1030450097C2A2C2A1E5B5547FF5B5E5B554BFF564
:10305500B5A220B34008E5B54404F5B58006E5B54D
:1030650054FBF5B5A20FB3500EE53AD394334007A0
:10307500E53AC394CC400302310BE5B54401F5B5FF
:10308500744690007EF090008AE075F064A4FFAE6F
:10309500F08E358F367402BE000AD39F4006753612
:1030A5000275350075A71085F95085FA517E017FA7
:1030B50000E55112520DE5502FFF50010E8E338F52
:1030C50034AC35AD36EF2DFDEE3CFC8C358D36D26E
:1030D50093D294D291D292D287E536F5FBE535F5B8
:1030E500FCE536F5E9E535F5EAE536F5EBE535F5E3
:1030F500ECE536F5EDE535F5EEE536F5FDE535F5C9
:10310500FE75A700D20FE53AC3941A5002C20F907C
:10311500001474FFF0A374DCF09000B1E090001A85
:10312500F8E4F0E8A3F0C213C215C21774C8900002
:1031350030F074C8900034F074C8900038F074C84A
:1031450090003CF0C210C211752600752500753C33
:1031550000C208756C00900022E4F0A3F0754C1EC7
:103165009007C0E0FEA3E0FF740312520D74011234
:1031750051FF9007BEEEF0A3EFF09000A3E06005CD
:103185001249BB8002C2049000A6E06005124AAB5A
:103195008002C206A204300501B35017A204B34051
:1031A50008E5B54408F5B58006E5B554F7F5B5A2CB
:1031B500049205A206300701B35017A206B34008D2
:1031C500E5B54402F5B58006E5B554FDF5B5A206AD
:1031D5009207C203752C00752B0090001CE4F0A328
:1031E500F0900092E075F032A4FFAEF090002AEE68
:1031F500F0A3EFF0900018E4F0A3F0C22190007F57
:10320500E0C3943C5019758D31758B00753D02E511
:103215004BB4090990007FE004F0754B00803BE555
:103225004BB40903754B00752800752700758D0093
:10323500758B00753D0090007EE0C3946450089046
:10324500007EE004F08006746490007EF090007EBD
:10325500E0B46406E5B554FEF5B5E543C3944150C5
:0D32650009740E90005BF0120579020D1443
:104FA5000000010001400160018001A001C001E095
:104FB50002000300039603B603D603F404000500BC
:104FC50005180530054805600578059005A805C054
:104FD500060006140628063C066E068C00FF013FF7
:104FE500015F017F019F01BF01DF01FF02FF039503
:104FF50003B503D503F303FF04FF0517052F054785
:10500500055F0577058F05A705BF05FF061306276D
:10501500063B066F068B06A9DAD8D7D5D4D2D0CFF2
:10502500CDCBC9C7C6C4C2C0BEBCBAB8B5B3B1AF93
:10503500ADABA8A6A4A2A09D9B99969492908D8BAA
:1050450089878482807E7C79777573716F6D6B69D2
:10505500676563615F5D5B5957565452504F4D4BC1
:105065004A4847454442413F3E3C3B3A393736354D
:10507500343231302F2E2D2C2B2A29282726252571
:105085002423222121201F1E1E1D1C1C1B1A1A1938
:1050950019EEECEBEAE9E8E7E5E4E3E1E0DEDDDB88
:1050A500D9D8D6D4D2D0CECCCAC8C6C3C1BFBCBA53
:1050B500B7B5B2B0ADABA8A5A3A09D9B98959290AE
:1050C5008D8A8785827F7D7A7775726F6D6A68654F
:1050D50063615E5C5A575553514F4D4B49474543A4
:1050E50042403E3C3B393836353332312F2E2D2B5D
:1050F5002A292827262524232221201F1E1D1D1C81
:0A5105001B1A1A19181817161615B0
:10329000750B00750A00AE0AAF0BAC08AD09EDC3A3
:1032A0009FEC9E401674FF12007575CF01780B7469
:1032B0000126F6500418E436F650DB22900053E065
:1032C000B4AA1C900786E0B43C159007C6E0FEA3A4
:1032D000E0FFEF4E6009741EBE0004D39F5003024E
:1032E00033EA75360075350075F8099007C6E0FEBB
:1032F000A3E0FF74076F4E6006740E6F4E70067485
:103300003A900786F09007C6E0FEA3E0FF7408BE7F
:10331000001ED39F401A7E017F089007C6E0FCA3E1
:10332000E0FD1DBDFF011C1200038E338F34801F92
:103330009007C6E0FEA3E0FF74081252648F048E6B
:10334000057E017F08CDCCCD1200038E338F34AEC5
:1033500035AF36740CD39F74019E50030233E5A23F
:10336000F9B3407EE5364535700375A382AE35AFBF
:103370003674016F4E700375A300AE35AF3674021C
:103380006F4E700D9007C7E075F002A4FDACF08D94
:10339000A3AE35AF3674036F4E700375A300AE3520
:1033A000AF367403BE00039F5013AC33AD34ED2F22
:1033B000FFEC3EFE900082125234E0F5A3AE35AF32
:1033C00036EFB40B09EEB401057414120075AE3576
:1033D000AF36EFB40B07EEB4010375F80D78351274
:1033E000527402334F900053E4F022753600753565
:1033F0000075F8099007C6E0FEA3E0FF7408BE0060
:103400001ED39F401A7E017F089007C6E0FCA3E010
:10341000FD1DBDFF011C1200038E338F34801F90F1
:1034200007C6E0FEA3E0FF74081252648F048E0505
:103430007E017F08CDCCCD1200038E338F34AE35A4
:10344000AF367411D39F74019E500302351BA2F94D
:10345000B35003023518E5364535700375A3D2AE77
:1034600035AF3674016F4E700375A300AE35AF36BD
:1034700074026F4E700D9007C7E075F002A4FDACAA
:10348000F08DA3AE35AF3674036F4E700375A30095
:10349000AE35AF3674046F4E700375A300AE35AF12
:1034A0003674056F4E700375A300AE35AF367406E3
:1034B0006F4E700375A300AE35AF3674076F4E7054
:1034C0000375A300AE35AF3674086F4E700375A355
:1034D00000AE35AF367408BE00039F5016AC33AD56
:1034E00034ED2FFFEC3EFE90007D125234E5A3F048
:1034F00075A300AE35AF36EFB41009EEB401057414
:1035000014120075AE35AF36EFB41007EEB40103F8
:1035100075F80D783512527402343E2275360075F6
:10352000350075F809AE35AF367417BE0004D39F69
:1035300050030235F4A2F9B350030235F1E53645E4
:1035400035700375A3D2AE35AF3674016F4E70037C
:1035500075A300AE35AF3674026F4E700D9007C77D
:10356000E075F002A4FDACF08DA3AE35AF36740368
:103570006F4E700375A300AE35AF3674046F4E7096
:103580000375A300AE35AF3674056F4E700375A397
:1035900000AE35AF3674066F4E700375A300AE35BE
:1035A000AF3674076F4E700375A300AE35AF367437
:1035B000086F4E700375A300AE35AF367408BE00B9
:1035C000039F500C900067125234E5A3F075A300DE
:1035D000AE35AF3674166F4E70057414120075AEAA
:1035E00035AF3674166F4E700375F80D783512527C
:1035F0007402352522900053E0B4AB0280030236FA
:103600008F75360075350075F809AE35AF36741212
:10361000BE007CD39F4078A2F9B34070E5364535B3
:10362000700375A382AE35AF3674016F4E700375AB
:10363000A300AE35AF3674026F4E700D9007C7E031
:1036400075F002A4FDACF08DA3AE35AF3674036FF8
:103650004E700375A300AE35AF367403BE00039FF2
:10366000500990006C125234E0F5A3AE35AF3674B9
:10367000116F4E70057414120075AE35AF367411AB
:103680006F4E700375F80D783512527402360A22A7
:1036900090005CE4F074649007C6F8E4F0E8A3F0EE
:1036A00012351C74C89007C6F8E4F0E8A3F0900047
:1036B00073E0B4371A900070E0900067F0900071EA
:1036C000E0900068F0900072E0900069F080469011
:1036D000005C7401F074659007C6F8E4F0E8A3F0AC
:1036E00012351C74C89007C6F8E4F0E8A3F0900007
:1036F00073E0B4371A900070E0900067F0900071AA
:10370000E0900068F0900072E0900069F08006742C
:103710000290005CF090005DE4F074669007C6F8DB
:10372000E4F0E8A3F012351C74C89007C6F8E4F082
:10373000E8A3F0900072E0B43712900070E09000BF
:1037400061F0900071E090006AF0807690005D7406
:1037500001F074679007C6F8E4F0E8A3F012351C96
:1037600074C89007C6F8E4F0E8A3F0900072E0B4E3
:103770003712900070E0900061F0900071E09000CE
:103780006AF0803E740290005DF074689007C6F89D
:10379000E4F0E8A3F012351C74C89007C6F8E4F012
:1037A000E8A3F0900072E0B43712900070E090004F
:1037B00061F0900071E090006AF080067403900060
:1037C0005DF022E55D2534FFAE3350010E9000869A
:1037D000125234E0F55EE55D2534FFAE3350010E44
:1037E0000FBF00010E900086125234E0F55F856530
:1037F00061E55EB55F05855E5D8041E55FD3955E01
:10380000401DE55FC3955E8560F0A4FFAEF0E56105
:103810008E048F05FF120085ED255EF55D801DE5A8
:103820005EC3955F8560F0A4FFAEF0E5618E048F06
:1038300005FF120085EDF404255EF55D22E55FD3FA
:10384000955E401DE55FC3955E8560F0A4FFAEF018
:10385000E5618E048F05FF120085ED255EF55D8024
:103860001DE55EC3955F8560F0A4FFAEF0E5618E57
:10387000048F05FF120085EDF404255EF55D22E559
:103880003875F00484FF7E008F5DE53875F00484A0
:10389000ADF07C008D60756504753301753400E50D
:1038A0005DC3943F50051237C380069001C5E0F513
:1038B0005D855D53755200900058E075F020A4FFBF
:1038C000AEF09000D7E08E048F05FF1200858D5D6D
:1038D0009000BFE0D3953850030239859000E3E0B3
:1038E000D395384010ED9001C6125249E0F5557558
:1038F00054000239829000AEE0D395384043E55D34
:103900009001C6125249E0F55EE55D9001E6125263
:1039100049E0F55F9000E3E0F4042538F56090009D
:10392000AEE0FE9000E3E0F4042EF561E55EB55FE5
:1039300005855E5D800312383D855D5575540080B8
:1039400041E55D9001E6125249E0F55EE55D9002C9
:1039500006125249E0F55F9000AEE0F4042538F518
:10396000609000BFE0FE9000AEE0F4042EF561E54B
:103970005EB55F05855E5D800312383D855D5575DA
:103980005400023A2C9000E6E0D395385011E55DE2
:10399000900246125249E0F555755400023A2C90B7
:1039A00000AFE0D395385043E55D900226125249AE
:1039B000E0F55EE55D900246125249E0F55F900049
:1039C000AFE0F4042538F5609000E6E0FE9000AF2B
:1039D000E0F4042EF561E55EB55F05855E5D80036C
:1039E00012383D855D557554008041E55D900206B5
:1039F000125249E0F55EE55D900226125249E0F56B
:103A00005F9000BFE0F4042538F5609000AFE0FE61
:103A10009000BFE0F4042EF561E55EB55F05855EBC
:103A20005D800312383D855D55755400229000F786
:103A3000E0F562756511753302753400AE25AF2669
:103A4000E56275F00FA4FDACF0EDD39FEC9E402134
:103A5000E5628E048F05FF120085ED75F010A4FF5E
:103A6000AEF0E53875F01184FD7C00ED2FF5638034
:103A70000EE53875F01184FF7E00EF24F0F56385C4
:103A8000635DE53875F01184AFF07E008F6012370A
:103A9000C3855D64AE25AF269000F7E075F00FA4F6
:103AA000FDACF0EDD39FEC9E4028753302753410C9
:103AB00085635D1237C385645E855D5FAE25AF2685
:103AC000E5628E048F05FF1252288D6085626112B7
:103AD000383D855D537552007555647554002290CC
:103AE00000F7E0F562756511753302753400AE2597
:103AF000AF26E56275F00FA4FDACF0EDD39FEC9E10
:103B00004021E5628E048F05FF120085ED75F010EF
:103B1000A4FFAEF0E53A75F01184FD7C00ED2FF5C1
:103B200063800EE53A75F01184FF7E00EF24F0F516
:103B30006385635DE53A75F01184AFF07E008F60B8
:103B40001237C3855D64AE25AF269000F7E075F0AF
:103B50000FA4FDACF0EDD39FEC9E402875330275A9
:103B6000341085635D1237C385645E855D5FAE2565
:103B7000AF26E5628E048F05FF1252288D608562A4
:103B80006112383D855D537552009000C1E0B40468
:103B900053E53875F00484FF7E008F5DE53875F0DD
:103BA0000484ADF07C008D60756504753301753457
:103BB00000E55DC3943F50051237C380069001C5F0
:103BC000E0F55DAE52AF53E55D12520D74648E04A4
:103BD0008F05FF120085AE52AF53EF2DFDEE3CFC7A
:103BE0008C528D537555647554002290008CE0B44E
:103BF0000146E54075F00584FF7E008F5DE5407568
:103C0000F00584ADF07C008D607565057533057534
:103C10003400E55DC3941750051237C38006900544
:103C20009DE0F55DAE54AF55E55D2FFF50010E747C
:103C3000641252648E548F5590008DE0B40146E5B5
:103C40004175F00584FF7E008F5DE54175F00584C8
:103C5000ADF07C008D60756505753305753448E5FC
:103C60005DC3941750051237C380069005E5E0F553
:103C70005DAE54AF55E55D2FFF50010E74641252D6
:103C8000648E548F5590009CE0B40249E543C39480
:103C90004175F00584FF7E008F5DE54375F0058476
:103CA000ADF07C008D60756505753306753400E5F3
:103CB0005DC3941350051237C38006900699E0F552
:103CC0005DAE54AF55E55D2FFF50010E7464125286
:103CD000648E548F559000DEE0B402028003023DF2
:103CE0008AE53875F01584FF7E008F5DE53875F044
:103CF0001584ADF07C008D607565157533037534E2
:103D0000F4E55DC3940B50051237C380069004851B
:103D1000E0F55DE55D75F0FFA4FFAEF09000DFE03B
:103D20008E048F05FF120085ED900081F0E53F7550
:103D3000F078A4FFAEF074FF8E048F05FF120085AB
:103D40008C338D3474028C068D071251FF8F5DAC5D
:103D500033AD347404FF1252288D607565047533D9
:103D60000675346EE55DC3941D50051237C3800699
:103D7000900711E0F55DAE54AF55E55D2FFF5001A2
:103D80000E74641252648E548F5522900094E0B4E5
:103D900001179007CBE02555FFAE5450010E90005F
:103DA000E8E01252648E548F55900094E0B40316EC
:103DB000A201B3B35010900080E0C39405A825B8C9
:103DC00000069526400280109000B6E02555FFAE13
:103DD0005450010E8E548F5590008EE0B402028034
:103DE00003023FB8900091E0602FE540D3941E405D
:103DF0002890001CE0FEA3E0FF9000CCE075F003EB
:103E0000A4FDACF0EFD39DEE9C400E9000F0E0A836
:103E100025B80005D395265003023FB89000D9E09D
:103E20008538F0A4FFAEF0740512520D74071251DC
:103E3000FF8E338F34900098E0A825B800049526B3
:103E40005012900099E075F002A4FDACF0EFC39D14
:103E5000EE9C4003023FB8E53875F00B84FF7E000E
:103E6000900616125234FEE0FFEE900090E0FEEF56
:103E70008E0088F0A4FFAEF074648E048F05FF12EC
:103E800000858C338D34900058E075F018A4FFAE97
:103E9000F09000D7E08E048F05FF1200858C068D10
:103EA0000790062E125234AE33AF34E012520D7426
:103EB000648E048F05FF1200858C338D34E53EA897
:103EC00033B80077D395344072E53EC39534FFE4B0
:103ED0009533FE8E338F347428BE00039F500C75CB
:103EE0003428753300740D90005BF0AE33AF34901E
:103EF0000091E012520D74288E048F05FF12008588
:103F00008C338D34AE52AF53740A8E048F05FF127A
:103F100000858D068C07AC33AD34CFCECF120003B5
:103F2000740A8E048F05FF1200858C338D34AE52D7
:103F3000AF5312526C8E528F53807DE53EA833B83A
:103F4000000495345072AE33AF34E53E1252648EA5
:103F5000338F347428BE00039F500C75342875339A
:103F600000740D90005BF0AE33AF34900091E0121E
:103F7000520D74288E048F05FF1200858C338D340A
:103F8000AE52AF53740A8E048F05FF1200858D0662
:103F90008C07AC33AD34CFCECF120003740A8E043D
:103FA0008F05FF1200858C338D34AE52AF53EF2D49
:103FB000FDEE3CFC8C528D5322AE52AF53AC54AD4F
:103FC0005512000374648E048F05FF1200858C5215
:103FD0008D53900089E08C068D0712520D74648E0B
:103FE000048F05FF1200858C528D53A2084017AE36
:103FF00025AF267405BE00039F5002D208E53AD3D0
:1040000094CC4002D2029000EBE0B402089000EDA4
:10401000E0640160028017AE52AF53E54412520DC6
:1040200074E78E048F05FF1200858C528D5390002B
:10403000ABE05402601B9000A2E0A825B80012D3A8
:104040009526400DA208B3B35007E53AC3949A40B1
:10405000028028AE5BAF5C9000A0E075F002A4FD8A
:10406000ACF0EF2DFDEE3CFC74022DFD50010CE593
:104070003ABC0007D39D4003756901853A5C755BC6
:1040800000E569700302410F9000FEE0C3956940AE
:1040900070E54075F00584FF7E009005861252346D
:1040A000E0F534753300AE33AF349000B0E0125217
:1040B0000D74648E048F05FF1200858C358D36904B
:1040C00000FEE004C395698C068D0712520D900026
:1040D000FEE08E048F05FF1200858C358D36900032
:1040E000A1E08C068D0712520D740A8E048F05FF15
:1040F000120085AE52AF53EF2DFDEE3CFC8C528D7D
:104100005305699000FEE0C39569500375690090FE
:1041100000ABE05401601B90009FE0A825B800129E
:10412000D39526400DA208B3B35007E538C394CC0D
:104130004002802590009DE075F003A4FFAEF0E5FD
:10414000662FFF50010E74032FFF50010EE538BE9D
:104150000007D39F4003756A01853866E56A7003DE
:104160000241EA9000FFE0C3956A4070E54075F0B7
:104170000584FF7E00900586125234E0F5347533D5
:1041800000AE33AF349000B0E012520D74648E0470
:104190008F05FF1200858C358D369000FFE004C33B
:1041A000956A8C068D0712520D9000FFE08E048FE9
:1041B00005FF1200858C358D3690009EE08C068DB3
:1041C0000712520D740A8E048F05FF120085AE523D
:1041D000AF53EF2DFDEE3CFC8C528D53056A9000E1
:1041E000FFE0C3956A5003756A009000B0E0A852E2
:1041F000B80004955350099000B0E0F55375520093
:10420000229000ECE0B40102800302430CA208B348
:10421000500302430A9000B7E0B40168AE52AF53B6
:10422000AC25AD26120003743C8E048F05FF1200EE
:10423000859000C7E0BC00109D400D9000C9E0A82B
:1042400052B8000495535002D203AE52AF53AC257E
:10425000AD26120003743C8E048F05FF120085907A
:1042600000C7E0C3940ABC0015D39D40119000C95B
:10427000E0C39405A852B80005D3955350028002BC
:10428000C2038068AE52AF53AC25AD261200037452
:10429000788E048F05FF1200859000C7E0BC0010E7
:1042A0009D400D9000C9E0A852B8000495535004F9
:1042B000D2038038AE52AF53AC25AD261200037442
:1042C000788E048F05FF1200859000C7E0C3940A22
:1042D000BC0015D39D40119000C9E0C39405A852BD
:1042E000B80005D3955350028002C203A203B34025
:1042F00019AE52AF539000C8E012520D74648E0490
:104300008F05FF1200858C528D538002C2039000EE
:10431000ECE0B40258E53875F00884FF7E008F5D4C
:10432000E53875F00884ADF07C008D607565087522
:1043300033017534E0E55DC3943F50051237C38007
:1043400006900285E0F55DE55D75F05EA4FFAEF0D8
:10435000740A8E048F05FF1200858C568D577402E7
:10436000BC000AD39D4006755702755600A200B3E3
:104370004006A202B3B35009900022E4F0A3F080FB
:1043800024AE52AF537400D39F74019E400C900032
:1043900022E552F0A3E553F0800B74FF900022F861
:1043A000E4F0E8A3F09000CEE0D394024006A20827
:1043B000B3B34002800DAE52AF53740212520D8E51
:1043C000528F539000B7E0B4010DAE52AF53740258
:1043D00012520D8E528F53AE52AF53745E12520D65
:1043E000740A8E048F05FF1200858C528D5374025F
:1043F000BC000AD39D400675530275520090002000
:10440000E552F0A3E553F022900058E090038612A5
:104410005249E0F567756864900058E0FE9000C26C
:10442000E0D39E4037E53875F00884FF7E008F5D4D
:10443000E53875F00884ADF07C008D607565087511
:104440003303753496E55DC3941F50051237C3805E
:104450000690043BE0F55D855D688035E53875F0D4
:104460000884FF7E008F5DE53875F00884ADF07C30
:10447000008D607565087533037534B6E55DC394CA
:104480001F50051237C3800690045BE0F55D855D23
:1044900068229000F8E0F562756511753304753493
:1044A00000AE25AF26E56275F00FA4FDACF0EDD3AC
:1044B0009FEC9E4021E5628E048F05FF120085ED82
:1044C00075F010A4FFAEF0E53875F01184FD7C00A6
:1044D000ED2FF563800EE53875F01184FF7E00EF57
:1044E00024F0F56385635DE53875F01184AFF07EE7
:1044F000008F601237C3855D64AE25AF269000F84B
:10450000E075F00FA4FDACF0EDD39FEC9E40287554
:10451000330475341085635D1237C385645E855D31
:104520005FAE25AF26E5628E048F05FF1252288DFF
:104530006085626112383D855D6775686422900010
:10454000F8E0F562756511753304753400AE25AF7A
:1045500026E56275F00FA4FDACF0EDD39FEC9E4014
:1045600021E5628E048F05FF120085ED75F010A421
:10457000FFAEF0E53A75F01184FD7C00ED2FF56398
:10458000800EE53A75F01184FF7E00EF24F0F563AC
:1045900085635DE53A75F01184AFF07E008F60129F
:1045A00037C3855D64AE25AF269000F8E075F00F47
:1045B000A4FDACF0EDD39FEC9E4028753304753418
:1045C0001085635D1237C385645E855D5FAE25AF80
:1045D00026E5628E048F05FF1252288D6085626188
:1045E00012383D855D677568649000F3E0B4047926
:1045F000900058E0FE9000C2E0D39E4037E5387549
:10460000F00884FF7E008F5DE53875F00884ADF01A
:104610007C008D60756508753303753496E55DC360
:10462000941F50051237C3800690043BE0F55D856A
:104630005D688035E53875F00884FF7E008F5DE5A4
:104640003875F00884ADF07C008D607565087533B1
:10465000037534B6E55DC3941F50051237C3800659
:1046600090045BE0F55D855D682290008CE0B4010C
:104670003BE54075F00584FF7E008F5DE54075F0F9
:104680000584ADF07C008D60756505753305753466
:1046900018E55DC3941750051237C380069005B521
:1046A000E0F55DE568255DC39464F56890008DE0F4
:1046B000B4013BE54175F00584FF7E008F5DE54167
:1046C00075F00584ADF07C008D607565057533056A
:1046D000753460E55DC3941750051237C3800690AA
:1046E00005FDE0F55DE568255DC39464F568E56763
:1046F0002568F55A900094E0B402109007CAE025AE
:104700005AFE9000E8E0F4042EF55A9000EBE0D356
:1047100094014040E544C394E7501D74E7C39544B9
:10472000FE9007CCE08E00F5F0E884FF7E008F5D00
:10473000E55A255DF55A801CE544C394E7FE9007D1
:10474000CCE08E00F5F0E884FF7E008F5DE55AC373
:10475000955DF55AA2084006E5672464F55AE55AC6
:10476000D394644009E55AC39464F55A8003755A9A
:10477000009000C4E0C3955A50069000C4E0F55A7A
:1047800022D2009000DAE0A825B800049526503B1C
:104790009000DAE0A825B8000495265003755A0F5A
:1047A0009000DAE004A825B8000495265003755A55
:1047B0000A9000DAE02402A825B8000495265005E6
:1047C000755A05C200740990005BF07E017F00906D
:1047D00000CAE012520D9000D9E08E048F05FF123E
:1047E0000085E538BC000CD39D4008C200740A90D7
:1047F000005BF09000CBE0C39540500D9000DDE0F1
:10480000A825B80006952640028008C200740B90C7
:10481000005BF0A2004003755A05900094E0B403D9
:1048200006A201B3B34002802B900080E0C3940540
:10483000A825B800049526500C9000B5E0F55A74F0
:104840000C90005BF0900080E0A825B8000495264D
:104850005002C200855A45900086E0255AFE90001D
:1048600058E075F01E84FC7F00EE2CF55A22900073
:1048700058E075F00584FF7E008F5D900058E0756C
:10488000F00584ADF07C008D6075650575330375AA
:1048900034D69000D7E01475F00584FF7E00E55D06
:1048A000BE00039F50051237C3800BE55D90045C8A
:1048B000125249E0F55DE55D9007CDF09007CDE03F
:1048C000FE9000C6E0C39E50089000C6E09007CD61
:1048D000F022E54075F00584FF7E009005861252B7
:1048E00034E0F56CE56CD394644010E56CC39464DB
:1048F00075F00F84FF7E008F6C8003756C00900054
:10490000A9E0256CF56C229007C0E0FEA3E0FF74DF
:10491000041251FFE53812520D740F8E048F05FFFB
:104920001200859007BEECF0A3EDF090009CE0B47F
:104930000262E543C3944175F00584FF7E008F5DFC
:10494000E54375F00584ADF07C008D6075650575F7
:104950003306753414E55DC3941750051237C380D0
:10496000069006ADE0F55D9007BEE0FEA3E0FF74A3
:104970000A8E048F05FF120085E55D8C068D0712F7
:10498000520D740A8E048F05FF1200859007BEEC4D
:10499000F0A3EDF09007BEE0FEA3E0FF9007C4E0B7
:1049A000FCA3E0FDEDD39FEC9E400F9007C4E0F820
:1049B000A3E09007BEC8F0A3C8F0229000A3E0B423
:1049C00001038526509000A3E0B402129000D9E0C4
:1049D0008538F0A4FFAEF074081251FF8F5090009C
:1049E000A3E0B40303853A509000A3E0B404038528
:1049F00040509000A3E0B40507E541C39414F5507E
:104A00009000A3E0B406038542509000A3E0B407F1
:104A1000038543509000A3E0B40803854450900000
:104A2000A3E0B40903853F509000A4E0FE9000A5E8
:104A3000E0D39E404B9000A3E0B404189000A5E0A2
:104A4000C395505002D2049000A4E0D39550400288
:104A5000C204802A9000A4E0C3955050099000A59C
:104A6000E0D3955050028002D2049000A4E0D39588
:104A70005050099000A5E0C395505002C204802A0E
:104A80009000A4E0D3955040099000A5E0C3955054
:104A900040028002C2049000A4E0C39550400990F7
:104AA00000A5E0D395504002D204229000A6E0B4C5
:104AB00001038526509000A6E0B402129000D9E0D0
:104AC0008538F0A4FFAEF074081251FF8F509000AB
:104AD000A6E0B40303853A509000A6E0B404038531
:104AE00040509000A6E0B40507E541C39414F5508A
:104AF0009000A6E0B406038542509000A6E0B407FB
:104B0000038543509000A6E0B4080385445090000C
:104B1000A6E0B40903853F509000A7E0FE9000A8EE
:104B2000E0D39E40409000A7E0C39550500990000C
:104B3000A8E0D3955050028002D2069000A7E0D39F
:104B4000955050099000A8E0C395505002C20690BD
:104B500000A6E0B401099000E5E0D3953A50028048
:104B600002C206802A9000A7E0D395504009900029
:104B7000A8E0C3955040028002C2069000A7E0C39F
:104B8000955040099000A8E0D395504002D20622EB
:104B9000AE58AF5974F5D39F74019E4008785812EF
:104BA0005274024C8B755901755800AE25AF26E53D
:104BB0006CBE000DD39F40099000BBE0D3956D40C3
:104BC00002801B756D00E56CC39526F5509000BE04
:104BD000E0D3956B4006E56B2550F56B8002056DC3
:104BE000900097E0D3953A401CE538D395394015AD
:104BF000AE25AF26E56CBE00039F50099000BCE0D7
:104C0000D3956E400280579007CEE0A825B80004E7
:104C1000952650037570009007CEE0A825B8000BCC
:104C2000D395264006E5269007CEF0E570702AE57C
:104C300026C3956CF550E550D39405400375500597
:104C40009000BDE0C3956B5007E550C3956B4002E3
:104C50008007E56BC39550F56B756E008002056E9D
:104C6000E5707016900097E0C3953A500DE56C24FE
:104C700005A825B8000695264002800F9000AAE0FE
:104C8000F56B75700174789007CEF022AE58AF596D
:104C900074E9D39F74039E40087858125274024EF0
:104CA00039755901755800756B32A222402A756B0F
:104CB000199000AAE075F002A4FFAEF0E56DBE0009
:104CC00006D39F4002D222056D7570037478900759
:104CD000CEF0756F00024E28AE25AF26E56C6F4E04
:104CE0007003024E28E56CBE000DD39F4009900072
:104CF000BBE0D3956D40028017756D00A208B3B379
:104D00005007E570C3940340028003756B19800D52
:104D1000E56CC39526F550E56D2550F56D9000972F
:104D2000E0D3953A400E9007CEE0A825B80007D30F
:104D300095264002800C056F9000AAE0B56F0375C0
:104D40007000E570B4030DE56C2402A825B80006D8
:104D500095264002800A056FE56FB43C037570022A
:104D6000E570B402299007CEE0A825B8000ED395CF
:104D7000264009E5269007CEF0756F00900097E079
:104D8000C3953A5009756F0074789007CEF0E570BE
:104D9000705A900097E0D3953A401CE538D3953986
:104DA0004015AE25AF26E56CBE00039F500990006C
:104DB000BCE0D3956E40028008756E00756B4B8029
:104DC00028E526C3956CF550E550D394054003754E
:104DD0005005900097E0D3953A4008E56E2550F5D0
:104DE0006E8006E56E2406F56E756F00E570701630
:104DF000900097E0C3953A500DE56C2405A825B8BE
:104E00000006952640028003757001E570B4011814
:104E1000756B19056F9000AAE0B56F067570027585
:104E20006F0074789007CEF0E56B75F00AA4FFAEC2
:0A4E3000F09007C8EEF0A3EFF022A7
:095249002582F582500205832242
:0F51F00025E050020583258250020583F58222B7
:10006400EF2F500205832582F582E5833E2EF5832A
:010074002269
:10526400CFC39FFF50011E22C3EF9DFFEE9CFE2281
:09525200E493F608740193F622BE
:085274000806B600021806222C
:0D521B00A3E004F0700612523FE004F02200
:0E003900A3E014F0B4FF0612523FE014F022D0
:0E51FF00048007C3CE13CECF13CFD5E0F62227
:10510F00BC000FBE0008ED8FF084FFADF022E4FE6F
:10511F00FF22BE000DEF60FE54F0606F20E7030228
:10512F0051C5EAC0E0EBC0E078017A0075F001EEFE
:10513F0020E710EF25E0FFEE33FE0AC5F023C5F0A0
:10514F0030E7F0EA5407F9096A7A007B006001083A
:10515F00C3EC9E40167004ED9F4010ED9FFDEC9E3A
:10516F00FCE5F0CA4ACA03F5F08005E5F003F5F057
:10517F00C3EE13FEEF13FFD9D77908CACBCAD8D025
:10518F00EAFEEBFFD0E0FBD0E0FA22EC8FF084FCDC
:10519F00ED54F045F0C48FF084FEEDC454F045F0AB
:1051AF00C48FF084FDEEC4FE54F02DFFEE540F3C7F
:1051BF00FEADF07C0022790078008FF0EC7E0820A5
:1051CF00E70DC3CD33CD33C933C9C833C8DEF0843F
:1051DF0049F9E5F08FF0BE00E6FD7C00E9FFE8FE3F
:0151EF00229D
:0E520D00F88FF0A4FFE5F0CE88F0A42EFE226C
:10000300EF8DF0A4F9A8F0EF8CF0A428F8EE8DF0B2
:06001300A428FEE9FF2213
:10007500600D782B02007F007830D8FED5E0F8229D
:10008500EEC0E07E0012510FEFFDEEFCD0E0FE2247
:0C522800EEC0E07E0012510FD0E0FE222C
:03001B0002001EC2
:03009B0002004917
:0300000002525B4E
:09525B0075817175D00002068610
:10523400E5822FF582E5833EF583220582D582023D
:05524400158315822214
:10001E00C0E0C0F0C083C082C0D075D000120653BD
:0B002E00D0D0D082D083D0F0D0E032E0
:10004900C0E0C0F0C083C082C0D075D0001206568F
:0B005900D0D0D082D083D0F0D0E032B5
:00000001FF
